:1000000012C019C017C016C015C014C013C012C04A
:1000100011C010C00FC00EC00DC00CC00BC00AC074
:1000200009C008C007C011241FBECFE5D4E0DEBF61
:10003000CDBFA4C0E5CF1FB6E0E6F0E079E10CC08B
:1000400035E13A95E1F040B34470D9F70000000083
:1000500000000000000000003ED0909A40B390984D
:10006000447041937A9539F035E13A9541F040B3C7
:100070004470D9F3E5CFE0E6F0E086803AC030E1A5
:10008000371B21F5E0E6F0E031913323F9F43191AB
:1000900031913323D9F431913323C1F43191332396
:1000A000A9F43191332391F43191332379F43191CF
:1000B0003323889409F00894E0E6F0E03191308130
:1000C000332311F018F410C008F009C01FBE1895B2
:1000D00033941FBE189533E03A95F1F70895EBE39A
:1000E000F1E078E114D0F2CFE3E5F1E070E50FD074
:1000F000EDCF662019F4E9E7F0E002C0E9ECF0E0AA
:10010000882011F070E501C070E401D0E1CF319199
:100110003323C9F400008A9A4FE04A95F1F70000B2
:100120008A9842E04A95F1F77A9589F70000000035
:1001300000000000000000008A9A44E04A95F1F7B0
:1001400000008A9808958A9A44E04A95F1F70000E1
:1001500000008A984CE04A95F1F7000000007A957B
:10016000B1F60000000000000000000000008A9AC4
:1001700044E04A95F1F700008A980895002407EEBC
:1001800005BB00E304BB0FEF08BB00E007BB0AEFB1
:1001900002BB01E001BB02E005BF00E40BBF42D19E
:1001A00010D119D15FD166243324F7D020D0552344
:1001B000E1F77724C9E1D1E00A85002311F001E0DD
:1001C000702A0B85002311F002E0702A0E810023B3
:1001D00011F004E0702A0F81002311F008E0702A6A
:1001E00078943320F1F303D000C03324FACFC9E16F
:1001F000D1E001E0099209920992099209920992CB
:10020000099209930993C9E1D1E009E0F02E37D1B1
:10021000FF2049F00895662019F4C9ECD0E0089554
:10022000C9E7D0E00895A9E1B1E0F5DF0D910F83B2
:100230000D910E830D9170FE098770FC0B870D9157
:100240000B830D910C870D910D870D910F870D91EB
:100250000E8712960D9170FE0B8770FC09870D9129
:100260000A8771FE09C0A9E1B1E01E960C910C83CA
:100270001E971F960C910D830985FF24002309F01A
:10028000F09418E0E096F9921A95E9F7C4DF0A8530
:10029000FF24002309F0F09418E0E896F9921A95EB
:1002A000E9F7A9E1B1E0B7DF1C960C91002341F416
:1002B000A9E1B1E01D960C91002321F40FE703C0E2
:1002C0000FEF01C000E010E8A896F12EF022F9929D
:1002D0001695D9F771FC19C0A9E1B1E09CDF1E9613
:1002E0000C91002341F4A9E1B1E01F960C91002389
:1002F00021F40FE703C000E001C00FEF10E8A09663
:10030000F12EF022F9921695D9F7A9E1B1E05096B5
:1003100014D072FE22D010E821277DDF609616D01F
:10032000A9E1B1E0589609D072FE17D010E8212754
:1003300072DF68960BD060940895222710E80D9123
:10034000002309F0212B1695D1F7089510E8F12E1E
:10035000F222F9921695D9F7089573FE04C0022F80
:100360000595020F07C0022F05950595102F1595CD
:10037000020F010F00231AF022233AF009C02223B2
:100380000AF406C00FE7202F04C000E8202F01C0A8
:10039000202F0EE10A95F1F708951F9317E60FEF4E
:1003A00000000000000000000000000000000A95AE
:1003B000B9F700000000000000001A9581F71F91B6
:1003C000089531E0EBE3F1E03496308333963083E7
:1003D0003B963083089531E0E3E5F1E038963083D1
:1003E00038963083369631933083329631933193F9
:1003F0003193308332963083329630833796308310
:1004000032963193319331933193319330833596D2
:1004100030833296319330833596308333963193DF
:10042000308308954427EBE3F1E038E141933A95B6
:10043000E9F7E3E5F1E030E541933A95E9F7E9EBD7
:10044000F0E0C9E0D1E030E1419349933A95E1F71A
:10045000E9EBF0E0C9E0D1E00FEF078307870F83F6
:100460000F870895A9ECB0E0E9E7F0E0C3E5D1E03B
:1004700000E4499141934D930A95D9F70895099164
:10048000002369F40000A39A1FE01A95F1F7000019
:10049000A39812E01A95F1F7FA9489F70EC0A39A7F
:1004A00014E01A95F1F700000000A3981CE01A95DB
:1004B000F1F700000000FA9411F755275095C9E1B3
:1004C000D1E021E205E10A95F9F013B31870D9F7EC
:1004D00000000000000000000000000011D0909A11
:1004E00013B39098187019932A9539F005E10A957D
:1004F00059F013B31870D9F3E5CFFF2455270895A9
:1005000003E00A95F1F70895FF24F39455275095D9
:0205100008954C
:00000001FF
